:100000000C94C1020C9405030C9405030C94050395
:100010000C9405030C9405030C9405030C94050340
:100020000C9405030C9405030C94B2140C948415E1
:100030000C94E6220C9405030C9405030C94050320
:100040000C9405030C9467030C9405030C940503AE
:100050000C9405030C944E230C9405030C94050397
:100060000C9405030C9405030C9405030C940503F0
:100070000C9405030C9405030C9405030C940503E0
:100080000C94270B0C9405030C9405030C940503A6
:100090000C9405030C9405030C9405030C940503C0
:1000A0000C9405030C9405030C940503F115131629
:1000B00001171316011758167B160117D016E316F1
:1000C000CD19CD19FC19FC193B1A5B1AB11BB11BD8
:1000D000661AB11B161B161B7D1B861BB11BAB1BA7
:1000E000231B231B231B231B231B231B231B231B20
:1000F000231B231B231B231B231B231B231B231B10
:10010000331B411B481B4F1B591B07634236B79BD0
:10011000D8A71A39685618AEBAAB558C1D3CB7CC67
:100120005763BD6DEDFD753EF6177231BF000000DF
:10013000803F08000000BE922449123EABAAAA2AC2
:10014000BECDCCCC4C3E00000080BEABAAAAAA3EDD
:1001500000000000BF000000803F00000000000819
:100160004178D3BB4387D1133D190E3CC3BD4282B6
:10017000AD2B3E68EC8276BED98FE1A93E4C80EF74
:10018000FFBE01C4FF7F3F00000000000000000030
:1001900000000000000000010204060A0F17202CD6
:1001A0003A4A5D71879DB3C7DAE9F5FCFFFCF5E9D2
:1001B000DAC7B39D87715D4A3A2C20170F0A0604EF
:1001C00002010000000000000000000029001400EF
:1001D0001A000800150017001C0018000C0012007F
:1001E00013002A002B0004001600070009000A0073
:1001F0000B000D000E000F0033003400E1001D0065
:100200001B00060019000500110010003600370021
:1002100038002872E000E200E300025403522C0090
:100220002C0004525000510052004F0029001400CD
:100230001A00090013000A000D000F0018001C002E
:1002400033002A002B0004001500160017000700D9
:100250000B00110008000C0012003400E1001D002A
:100260001B000600190005000E00100036003700C4
:1002700038002872E000E200E300025403522C0030
:100280002C0004525000510052004F000100420067
:100290004300440045004B002202380024002500A2
:1002A00026002A0001003E003F00400041004E00B1
:1002B0004A002502210022002300310201003A00F9
:1002C0003B003C003D004C004D0027001E001F007D
:1002D00020000100010001000100010001000100F7
:1002E000010001005000510052004F0035021E0273
:1002F0001F022002210222022302240225022602DA
:1003000027022A0001003A003B003C003D003E006D
:100310003F002D022E022F02300231020100400068
:1003200041004200430044004500005301530030A7
:100330000050010001000100010001000100010066
:1003400001000100AB00AA00A900AE0035001E00AC
:100350001F00200021002200230024002500260089
:1003600027002A0001003A003B003C003D003E000F
:100370003F002D002E002F00300031000100400012
:100380004100420043004400450000530153003047
:100390000050010001000100010001000100010006
:1003A00001000100AB00AA00A900AE002803540020
:1003B00068006500200050006C0061006E00630062
:1003C0006B0020004B006500790062006F00610047
:1003D0007200640000002C034F007200740068007B
:1003E0006F006C0069006E00650061007200200003
:1003F0004B006500790062006F00610072006400CC
:10040000730000000403090409026D00040100A048
:10041000FA09040000010301010009211101000192
:10042000223F000705810308000A090401000103B7
:10043000010200092111010001224D00070582037C
:1004400008000A090402000103000000092111014B
:1004500000012236000705830308000A090403008F
:1004600001030000000921110100012239000705E4
:1004700084031000011201100100000008EDFE606D
:100480006001000102000105010906A1010507192B
:10049000E029E71500250195087501810205081975
:1004A00001290595057501910295017503910105D5
:1004B000071900297715002501957875018102C07B
:1004C00005010980A101850216010026B7001A0165
:1004D000002AB700751095018100C0050C0901A123
:1004E000018503160100269C021A01002A9C027550
:1004F0001095018100C005010902A1010901A100B7
:1005000005091901290515002501950575018102C7
:100510009501750381010501093009311581257F98
:1005200095027508810609381581257F95017508A2
:100530008106050C0A38021581257F950175088111
:1005400006C0C005010906A101050719E029E71544
:100550000025019508750181029501750881010545
:1005600008190129059505750191029501750391F9
:10057000010507190029FF150025FF95067508815B
:1005800000C011241FBECFEFDAE0DEBFCDBF04B63E
:1005900003FE24C080911E0390911F03A0912003AD
:1005A000B09121038730904BA740B04BB9F4109223
:1005B0001E0310921F03109220031092210314BEF9
:1005C00084B7877F84BF88E10FB6F894809360007A
:1005D000109260000FBEE0E0F8E3099511E0A0E0A2
:1005E000B1E0E6E2FAE502C005900D92A03CB10749
:1005F000D9F713E0A0ECB1E001C01D92AE31B10714
:10060000E1F70E94F8110C94112D0C94000008954C
:10061000089581E0089508950C9408030C9409034B
:100620000C940B030E94DB2823E030E0281B3109E7
:10063000220F2093C4010895282F2F9880918000C5
:10064000211108C0877F8093800010928D00109246
:100650008C001BC0886080938000233019F48FEFDA
:100660009FEF0FC083E090E0821B9109880F991FD4
:100670002FEF3FEFA90102C0569547958A95E2F703
:10068000CA0190938D0080938C000C9412030E94F9
:10069000120384E08093C3011092C0010895279A49
:1006A0002F988FEF9FEF90938700809386008AE0CA
:1006B0008093800089E1809381000E9444280C94FB
:1006C00047030E944F036E9A769A0C9407031F9279
:1006D0000F920FB60F9211242F933F938F939F93F6
:1006E000EF93FF93E091C101F091C201CF01019618
:1006F0009093C2018093C1010090C30102C0F6959E
:10070000E7950A94E2F7EF738091C001823019F403
:10071000E03251F404C0813039F4EF3329F4809190
:100720006F008D7F80936F00F0E0E457FE4FE491FF
:1007300021E031E0E29FC001E39F900D1124009081
:10074000C40102C0969587950A94E2F790938D00B4
:1007500080938C00FF91EF919F918F913F912F910A
:100760000F900FBE0F901F90189561110DC0FC01E6
:100770008281882331F085EE0E9471180E949B28A7
:1007800003C085EE0E94391980E090E0089581E071
:1007900008950C94C70308950C9461038091150289
:1007A000882309F448C08091D1019091D20100972B
:1007B00079F40E9418239093D2018093D101809103
:1007C000D30190E0009771F48091D40190E00AC0C9
:1007D0000E9424232091000130910101281739073C
:1007E00040F329C00197880F991F880F991FFC01BA
:1007F000EB52FE4F60817181828193810E948D0A4C
:10080000E091D30184E0E89FF0011124EB52FE4F08
:1008100060817181828193814FE050E00E94450E9A
:100820008091D30190E001966091D40170E00E9424
:10083000C12C8093D3010C940C03109217020C94DA
:100840005A0A0895089581E0809317020C942204B7
:10085000089508958F929F92AF92BF92EF92FF9268
:100860000F931F93CF93DF93CDB7DEB7A3970FB648
:10087000F894DEBF0FBECDBF7C01FC010081118169
:10088000C8010E941521B8010E942C068C01B701F5
:100890000E94C903882309F4CCC10032F0E51F0788
:1008A00041F4F7018281882309F458C00E94A90EFF
:1008B000C0C10132F0E51F0741F4F70182818823AE
:1008C00009F44CC00E94B20EB4C10232F0E51F0719
:1008D00051F4F7018281882309F440C00E94A50EDB
:1008E0008111F0CFE3CF0332F0E51F0739F4F701B0
:1008F0008281882399F10E9423049BC10432F0E590
:100900001F0739F4F7018281882341F10E941D04F9
:1009100090C10532F0E51F0749F4F7018281882371
:10092000E9F0809117028111F1CFE5CF0632F0E5B1
:100930001F0739F4F7018281882381F00E94B90EE4
:100940000AC00732F0E51F0749F4F70182818823C6
:1009500029F00E94C40E0E9429046BC180911702E5
:10096000811105C0F70182818111CFC018C1003EFD
:10097000110579F4F7018281882309F44DC00E94A2
:100980005A0A81E080931602109215021092D40147
:1009900050C1023E110559F4F70182818823E1F12B
:1009A0000E945A0A109216021092150242C1033E8A
:1009B000110591F4F7018281882371F10E945A0A8E
:1009C0001092160281E0809315021092D3011092CA
:1009D000D2011092D1012DC10235110559F4F70150
:1009E0008281882309F425C1809100019091010141
:1009F0000A970DC00135110579F4F701828188232A
:100A000009F417C180910001909101010A96909319
:100A10000101809300010DC14091040183E2EFE1E7
:100A2000F1E0DE01119601900D928A95E1F7F70150
:100A3000808121E030E02C0F3D1F280F311DC901BE
:100A40002091020130910301FC01E20FF31F60814C
:100A5000772767FD7095640F711D882777FD809556
:100A6000982F0E94E32920E030E040E451E40E9406
:100A700048294B015C01F701218184E090E0821B51
:100A80009109BC01882777FD8095982F0E94E32962
:100A90009B01AC01C501B4010E94E0289B01AC019F
:100AA00060E070E080E090E40E94562B20E030E0AF
:100AB0004CED50E40E94F32A4B015C01F701828166
:100AC0008823D1F04FE050E0C501B4010E94450EEB
:100AD000809116028823A1F08091D40124E0829FA6
:100AE000F0011124EB52FE4F80829182A282B382E8
:100AF0008F5F8093D40104C0C501B4010E948D0AA8
:100B00000F3F110508F02ECF94C08091D0018111C4
:100B10001FC0043130E5130709F051C00E94CB0318
:100B200081E08093D0010E9418239093CF0180939D
:100B3000CE011092C7011092C9011092C801109203
:100B4000CB011092CA011092CD011092CC0171C05C
:100B50008091CE019091CF010E942423883C910581
:100B600070F48091C701E82FF0E0EE0FFF1FE8530B
:100B7000FE4F118300838F5F8093C7015AC00438F2
:100B800080E5180721F00538104501F13AC0F7015A
:100B90008281882341F01092C50182E01EC0043892
:100BA00030E5130759F58091C501811106C086E231
:100BB0000E94711886E20E94391982E01CC0043834
:100BC000F0E51F0741F305381045D9F4F70182819C
:100BD000882331F01092C60180E20E94881929C052
:100BE0008091C601811106C087E20E94711887E2D8
:100BF0000E94391980E20E948F191BC005381045E8
:100C000029F381E08093C5018093C601C701A396B3
:100C10000FB6F894DEBF0FBECDBFDF91CF911F910D
:100C20000F91FF90EF90BF90AF909F908F900C949A
:100C30000E0380E0A3960FB6F894DEBF0FBECDBFC3
:100C4000DF91CF911F910F91FF90EF90BF90AF90E8
:100C50009F908F90089508959CE0799FF001112452
:100C600090E3899FE00DF11D1124E60FF11DEE0FB9
:100C7000FF1FE453FE4F859194910895880F991FAB
:100C8000FC01E45BFF4F859194910895880F991FB3
:100C9000FC01E453FE4F8591949108950F931F93A7
:100CA000CF93DF93EC01811521E39207A0F5C115E5
:100CB00080E3D80708F0D7C0C83ED105D8F4C03EBD
:100CC000D10508F007C2C83AD10578F4C53AD10574
:100CD00008F06AC0C130D10509F463C008F4F7C157
:100CE000C430D10508F0F6C1F2C1CB3BD10508F400
:100CF00066C0EDC1C11590E2D90708F0AFC0C115BB
:100D000021E0D20708F0E6C1C03FD10508F4DFC1F9
:100D10008E0110651FC2C03880E5D80700F5C037C6
:100D200090E5D90708F0A3C0C11520E5D20709F462
:100D3000ACC050F4CE01905480319F4008F0C7C140
:100D4000DF708E01106A06C2C13080E5D80709F451
:100D5000AEC0C43190E5D90708F4AFC0B8C1C338FC
:100D600020E5D20709F48EC050F4C13890E5D907C8
:100D700009F482C008F083C000E011EDEBC1C0317E
:100D800081E5D80708F4A3C1C11597E5D90708F490
:100D900036C1CE0190578115904108F098C1DF709F
:100DA00093C101E010E0D6C1C53AD10509F494C160
:100DB000C63AD10509F093C102E810E4CBC1C83AA4
:100DC000D10509F48FC1C93AD10509F48EC1CA3AD7
:100DD000D10509F48DC1CB3AD10509F48CC1CC3AC7
:100DE000D10509F48BC1CD3AD10509F48AC1C03BC4
:100DF000D10509F489C1CE3AD10509F488C1CF3AA9
:100E0000D10509F487C1C13BD10509F486C1C23BB4
:100E1000D10509F485C1C33BD10509F484C1C43BA4
:100E2000D10509F483C1C53BD10509F482C1C63B94
:100E3000D10509F481C1C73BD10509F480C1C83B84
:100E4000D10509F47FC1C93BD10509F47EC1CA3B74
:100E5000D10509F47DC100E014E47CC1CE019F708E
:100E60000E94460678C1DD278E01106C73C1CF70D9
:100E7000DD278E01146D6EC100E010ED6BC100E046
:100E800012ED68C100E013ED65C10E941C1C0E94B8
:100E90005A0A0E9421048FEF94E32CE08150904085
:100EA0002040E1F700C000000E94732353C18091ED
:100EB000F20281608093F2024DC10E94D42381111D
:100EC00002C00E94B0230E94E72390E090931D038C
:100ED00080931C03C23080E5D80721F480911C0365
:100EE000816086C0C43090E5D90721F480911C034D
:100EF00082607EC0C63020E5D20721F480911C03B9
:100F0000846076C0C83080E5D80719F480911C034E
:100F100027C0CA3090E5D90721F480911C03806175
:100F200067C0CC3020E5D20721F480911C03806299
:100F30005FC0CE3080E5D80721F480911C03806427
:100F400057C0C03190E5D90721F480911C03806817
:100F50004FC0C23120E5D20729F480911C03846080
:100F6000886046C0C33080E5D80721F480911C0317
